:1000000000308A00FC2A0000831A0A288E00030EA2
:100010008F000F2883128E00030E8F008F148E0E18
:10002000040890000C0891000D08920083128B1EAA
:100030001B280B1978291008840011088C0012085D
:100040008D000F0E830083120E0E8F188316090089
:100050000A108A100A11033E020703188A0A820056
:10006000AA34C034B634C034BB344034DD34C03478
:10007000BA34C034D734C034BB34C034BF34403455
:10008000BF34C034EF340034E8340034DB34C034DF
:10009000B7344034F8340034DD344034EA34C0340A
:1000A000BD34C034BD344034EB344034EB34C03460
:1000B000D634C034DA34C034DB344034D534C034C0
:1000C000DE34C034DF344034ED34C034D534403411
:1000D000D7344034EE34C034BE34C034DF34C0349E
:1000E00080340034FF348034AF348034FA348034C8
:1000F000ED348034B5344034AE34C034BF34803451
:10010000FB340034F7340034B7348034EF348034B7
:10011000EA340034D4340034AE340034D73480347C
:10012000B7340034BD340034ED340034FF340034CF
:10013000BB348034AD348034B5348034D63480342C
:10014000D5348034DB348034F5340034DE3480340C
:10015000F6348034AA340034EB348034AB34C03409
:10016000AF344034FA340034EB340034AD3400346E
:10017000B5340034EE340034DB340034FD34003464
:10018000AA348034FE340034FE348034BE348034EB
:10019000D7340034BB340034DD340034AB340034A5
:1001A000D5340034EE348034AF340034DE340034DF
:1001B000DA340034AB348034DA348034AE34803412
:1001C000BA348034BD348034AB344034FB348034B2
:1001D000F7348034FD348034AF34C034B6348034E6
:1001E000B734C034B0340034BE340034BC340034CE
:1001F000B4340034C0340034F4340034B634003441
:10020000AC340034D0340034F5348034BF3400349E
:10021000D8340034EC340034F0340034E0340034AA
:10022000FC340034DF348034A8340034B834003473
:10023000A0340034DC340034F6340034D6340034D6
:10024000DF340034BA340034EA348034AD34C0349E
:10025000DD348034AD344034B534C034ED34403412
:100260000A148A100A1182071834183419341B34FE
:100270001D341E3421342334253428342A342C34BC
:100280002F3431343434363438343B343D34403414
:10029000423444344634483449344B344C344D347D
:1002A0004E344F344F344F340A148A100A118207E7
:1002B0005C345C3459345834563452344E344934F6
:1002C00043343D3435342E342634203416340D3442
:1002D0000534173420342834313439343E3444342E
:1002E00049344D345234543458345A345B345C34C9
:1002F00000000000273081001808990064309A003F
:1003000019089A02003065008515990B8529851119
:100310009A0B8829083065009C0A20301C02031CB7
:1003200093294D149C01061AA929861DA0291F3066
:100330001B020318A0299B0A1B0830219800A8293A
:100340009B080319A8291B089B031B083021980050
:10035000BB294D1AAD294D169B011B08542198004D
:100360001F301B020318BB299B0A13301B02031DFD
:10037000BB29043086060B118A111B2889018316BC
:10038000081483120808930000344F3084000008DA
:100390000319D92901308D00BF308C0064008C0B0B
:1003A000CE298D0BCC2927308C008C0BD529800BC6
:1003B000CA2900348B138B1BDA29FA30CF00C521F0
:1003C000FA30CF00C521FA30CF00C5210610CE1D6E
:1003D000861000340614861400344D1CF529CD19FE
:1003E000F329083086064D104D1500346400940141
:1003F000130814020318062ACD114D124D114D1980
:10040000042A6400ED21FF29940AF829003493138B
:100410001308960013089607160828209500CD1497
:10042000CF01CD154D174E198617CD1C3D2A6400FE
:100430004D114D13CD194D17CD11951BCD15CD1A5D
:10044000252ACD164D12CD194D16CF0A0310950D44
:100450004D1B2C2ACD1DCD1008304F02031C352A10
:10046000960A160828209500CF01CD124D193B2A77
:100470006400ED21362A8613152A003494011408ED
:10048000890083160814831208089300130A0319BD
:100490005E2A4030140203185E2A1408890083166D
:1004A00008148312080893000722940A140889008C
:1004B00083160814831208089300462A0034083073
:1004C0008C008316061783126400061F642ACF016E
:1004D0008C17782A8C13782A0310CF0C061FCF179D
:1004E0000C17782A0C138C0B6C2A4F088D00832A6A
:1004F000F2308C1B42308D008D0B7C2A8C1B6A2ABB
:100500000C1B722A6C2A642B930114081302031823
:10051000A82A640013081A0799001D3013078400E5
:100520000008CF00190889004F0888000B088C00CC
:100530008B138316081555308900AA30890088145A
:100540008818A02A081183120C088B00930A852AA8
:100550006400990A403019020318C32A1908890057
:10056000FF3088000B088C008B138316081555305C
:100570008900AA30890088148818BC2A08118312BF
:100580000C088B00640000349A0140301A020318F2
:10059000D62A1A08890083160814831208088C00CA
:1005A0000C0A0319D62A64009A0AC52A1A081407E5
:1005B0008C0040300C02031CDF2A4030940084225F
:1005C000872B8901130888000B088C008B13831676
:1005D000081555308900AA30890088148818EE2A39
:1005E000081183120C088B0000341D30140784009E
:1005F00013088000940A00348401830183160510D7
:10060000831205142730810001308C008C1D102BC3
:1006100007308101813084000008C0390F38800024
:100620006400813084000008C0390C0480008B16FF
:1006300081308400801300306500703066004D10FA
:10064000CD134E104E15CD100F309B004D13323090
:100650009800861AF42BBE2113088039003803193C
:10066000332BCE15342BCE116400DA219401CD1337
:100670004E10CE10CD1BCB2B01309A009901061BDA
:10068000612B64009A0A9A08031D482B990A9A0A5A
:10069000FE301902031D5D2B4E198617CE1D5C2BF3
:1006A0008613EA218B1750309300F62194013E22E5
:1006B000DA2101309A009901602B190A0319861377
:1006C0003F2B4E1986175F2A0D089300861393134C
:1006D000203013020318B72B033013020319B72B72
:1006E0001B3013020319B72B02301302031D7A2BA0
:1006F0009401B62B11301302031D822B9A01842220
:100700009401B62B12301302031D892BC42A9401C5
:10071000B62B13301302031D922BBE219317E12237
:10072000902BB62B14301302031D9B2BBE21931369
:10073000E122992BB62B0E301302031DA32BCD17EC
:10074000CE149401B62B0F301302031DA92B86146F
:10075000B62B17301302031DAF2B4E15B62B1830D6
:100760001302031DB52B4E11B62BF522B82BF52223
:1007700031301402031CBE2B1408940303301302FF
:10078000031DC42BCD17CA2B1B301302031DCA2B0C
:10079000CD17CE143A2BCD1FF32BEA218B17A030A7
:1007A0009300F6219401203093004E18ED2B1D305C
:1007B0001407840000089300940A033013020319FD
:1007C000E92B1B3013020319E92B31301402031CEF
:1007D000EB2B4E14EC2B0722D52B4E1CF12BCE1CF1
:1007E0003E224E18CD13FA2B8B17EA21503093007E
:0807F000F6213E22292B6300D3
:02400E00FD3F74
:104200000A000D0059006F007500720020006D005B
:10421000650073007300610067006500200067009F
:104220006F00650073002000680065007200650083
:104230002E0020004900740020006D00610079000C
:10424000200063006F006E007400610069006E0062
:10425000200075007000200074006F002000360000
:104260003400200063006800610072006100630098
:1042700074006500720073002E000A000D00FF003C
:00000001FF
